:020000040000FA
:040000006C303A28FE
:08000800A000030EA100831209
:1000100005191028831601178312B23081002B288E
:1000200083160113831203140B190310A80DA90DD5
:10003000AA0DAB0DAC0DAC16FF302C02031D2B2806
:10004000FA302B02031D2B2831152A08AF0029088E
:10005000AE002808AD008B100B11210E8300A00EFE
:04006000200E090065
:0C007400203084008001840A6030040207
:10008000031C3C281230B0008A218316FF23900005
:10009000831283160C308505870183128501870141
:1000A000073099000030831691008312C830831600
:1000B0008100831231309000003083168C0083124F
:1000C00010308B00831600309B001C141A0883121A
:1000D000BC00851DCE21831610309B001C141A080D
:1000E0008312BD00C62181018E018F010B118B107F
:1000F0000B108C018B178A2031198D20B30B8828A7
:10010000031085190314B90DF030390203190921C0
:10011000F3217B2864003210080031110130B70050
:100120008B132030370783169B001C141A08831288
:10013000A4001030370783169B001C141A08831282
:10014000A300A6000230A6060030370783169B00E6
:100150001C141A088312A200A7000130A7068B17EF
:10016000321CB82822090339A200A309A409A50951
:1001700024082F02031D032923082E02031D03292F
:1001800022082D02031D032901303702031DCD284B
:100190003D18CD283D143E14962102303702031D30
:1001A000D628BD18D628BD143E1498210330370236
:1001B000031DDF283D19DF283D153E149A21043028
:1001C0003702031DE828BD19E828BD153E149C21FF
:1001D00005303702031DF1283D1AF1283D163E1463
:1001E0009E2106303702031DFA28BD1AFA28BD16D3
:1001F0003E14A02107303702031D03293D1B0329AC
:100200003D173E14A221B70A083037020318080030
:1002100090280130B600B300B400B500B7008501E6
:100220008701B1138A20B30B3D29031085190314EC
:10023000B90DF030390203196429B40B3D2901309E
:1002400037020319AD21023037020319B2210330FE
:1002500037020319B521043037020319B8210530DC
:1002600037020319BD21063037020319C0210730B8
:1002700037020319C3219630B400311D1229311100
:10028000321C47292D090339AD00AE09AF092F1CD7
:1002900012298E018F010C1C12290C102E1E1229FE
:1002A0008B1320303707BB002F08BA00772110309E
:1002B0003707BB002E08BA00772100303707BB0094
:1002C0002D08BA0077218B1785018701B70AB6017F
:1002D00008303702031C1229C62108003E1C080002
:1002E0003E101030BB003D08BA00772108008B1388
:1002F0003A0883161C159A003B089B0055309D0058
:10030000AA309D009C1464009C1883291C11831240
:100310008B170800FF30D000D415D515D615D7158A
:10032000D815D915DA15DB15DC150800F130A5292B
:10033000F230A529F430A529F830A5291F30A929C4
:100340002F30A9294F30A9290800BD050F30D2044C
:100350000800BD05F030D2040800103085060230D8
:100360008706080020308506080021308506080031
:10037000023085060230870608001830870608001C
:100380002130870608000930870608003D08D200A2
:10039000031D08001130BD00D2000800B601B301F2
:1003A000B4013C1CD629BC01BC14D829BC013C14A6
:1003B0003C08B6006400DC29DD29DE29DF29E029BC
:1003C000B41B0516B41F0512B30BDA29B40BDA29D6
:1003D0000310B60CB608031DDA290030BB003C0838
:1003E000BA00772108008F08031908008F01D00F89
:1003F0002E2BD00A0E305205031D0D2A541D032A40
:10040000D40154161B2AD41D082AD40154161B2AC1
:10041000541E1B2AD401D4141B2AD41C122AD40122
:1004200054151B2A541D172AD401D4151B2A541EF7
:100430001B2AD401541509305205031D2E2A551DBF
:10044000242AD50155163C2AD51D292AD501551631
:100450003C2A551E3C2AD501D5143C2AD51C332AEA
:10046000D50155153C2A551D382AD501D5153C2AEC
:10047000551E3C2AD50155150B305205031D4F2A38
:10048000561D452AD60156165D2AD61D4A2AD60182
:1004900056165D2A561E5D2AD601D6145D2AD61C34
:1004A000542AD60156155D2A561D592AD601D6154D
:1004B0005D2A561E5D2AD601561507305205031DCA
:1004C000702A571D662AD70157167E2AD71D6B2A18
:1004D000D70157167E2A571E7E2AD701D7147E2AA7
:1004E000D71C752AD70157157E2A571D7A2AD7019E
:1004F000D7157E2A571E7E2AD7015715063052057A
:10050000031D912A581D872AD80158169F2AD81DE5
:100510008C2AD80158169F2A581E9F2AD801D81411
:100520009F2AD81C962AD80158159F2A581D9B2A05
:10053000D801D8159F2A581E9F2AD8015815103067
:10054000BC1819305205031DB42A591DAA2AD90115
:100550005916C22AD91DAF2AD9015916C22A591EC5
:10056000C22AD901D914C22AD91CB92AD9015915CC
:10057000C22A591DBE2AD901D915C22A591EC22A1A
:10058000D90159155030BC1859305205031DD72ACE
:100590005A1DCD2ADA015A16E52ADA1DD22ADA01C5
:1005A0005A16E52A5A1EE52ADA01DA14E52ADA1C77
:1005B000DC2ADA015A15E52A5A1DE12ADA01DA1590
:1005C000E52A5A1EE52ADA015A156030BC1869304E
:1005D0005205031DFA2A5B1DF02ADB015B16082B6E
:1005E000DB1DF52ADB015B16082B5B1E082BDB01EC
:1005F000DB14082BDB1CFF2ADB015B15082B5B1DC2
:10060000042BDB01DB15082B5B1E082BDB015B15C4
:100610002030BC1829305205031D1D2B5C1D132BE7
:10062000DC015C162B2BDC1D182BDC015C162B2B44
:100630005C1E2B2BDC01DC142B2BDC1C222BDC01A5
:100640005C152B2B5C1D272BDC01DC152B2B5C1E7A
:100650002B2BDC015C156E213D08D2005008D10027
:100660000C305405031D05120C305505031D851271
:100670000C305605031D05100C305705031D851061
:100680000C305805031D87100C305905031D071049
:100690000C305A05031D87120C305B05031D071231
:1006A0000C305C05031D871151080E020318802BC6
:1006B00012305405031D051612305505031D85160D
:1006C00012305605031D051412305705031D8514FD
:1006D00012305805031D871412305905031D0714E5
:1006E00012305A05031D871612305B05031D0716CD
:1006F00012305C05031D8715FF30500203190800F6
:100700008F08031D08008A2051080E02031C802B4D
:1007100018305405031D051206305405031D051637
:1007200018305505031D851206305505031D851625
:1007300018305605031D051006305605031D051417
:1007400018305705031D851006305705031D851405
:1007500018305805031D871006305805031D8714EF
:1007600018305905031D071006305905031D0714DD
:1007700018305A05031D871206305A05031D8716C7
:1007800018305B05031D071206305B05031D0716B5
:1007900018305C05031D871106305C05031D8715A5
:0207A00008004F
:084000000A00030002000600A3
:02400E00CC01E3
:10420000010078007A007C007E007B0079007F004E
:104210007D007A0078007E007C00FF00FF00FF0038
:104220000000F200F600FA00FE00F200F600FA00CC
:10423000FE00F200F600FA00FE00FF00FF00FF00A3
:10424000010005000500050005000900090009003E
:1042500009000D000D000D000D00FF00FF00FF0024
:10426000FF00FF00FF00FF00FF00FF00FF00FF0056
:10427000FF00FF00FF00FF00FF00FF00FF00FF0046
:10428000FF00FF00FF00FF00FF00FF00FF00FF0036
:10429000FF00FF00FF00FF00FF00FF00FF00FF0026
:1042A000FF00FF00FF00FF00FF00FF00FF00FF0016
:1042B000FF00FF00FF00FF00FF00FF00FF00FF0006
:1042C000FF00FF00FF00FF00FF00FF00FF00FF00F6
:1042D000FF00FF00FF00FF00FF00FF00FF00FF00E6
:1042E000FF00FF00FF00FF00FF00FF00FF00FF00D6
:1042F000FF00FF00FF00FF00FF00FF00FF00DD00E8
:00000001FF
